:020000001028C6
:10000800FE00030EF0000408F1000A08F200831253
:1000180003137F08F3007229672983120313A100D1
:10002800802180217908013A83120313A000200857
:10003800F9007908013A031D222823282528802160
:1000480027287D212728043083120313A0002008C5
:10005800A2002208FF3A031D3228332835285428E5
:1000680054287608840083130008A000220A3E283A
:100078000310A00CFF3E031D3C28201C44284528E3
:100088004728802149287D214928013083120313FC
:10009800A2022208FF3A031D522853283528542863
:1000A8000530A0002008A2002208FF3A031D5D28A1
:1000B8005E2860287F287F28210884008313000891
:1000C800A000220A69280310A00CFF3E031D672820
:1000D800201C6F2870287228802174287D2174289C
:1000E800013083120313A2022208FF3A031D7D2860
:1000F8007E2860287F284721080083120313A00068
:10010800A1010330F4007408A2002208FF3A031D7D
:100118008E288F289128DF28DF28FF3086000130BD
:10012800F400220A99280310F40DFF3E031D9728B6
:100138007408FF3AF500750886050430F400740861
:10014800A30008302302031CAA28AB28AD28D62810
:10015800D6280130F4007408A1070608F400230A21
:10016800B7280310F40CFF3E031DB5287418BD28EA
:10017800BE28CB282108F4002008840074088313C3
:1001880080000130AC000030AD00DF28DF280130EE
:10019800F4007408A30708302302031CD428D528C8
:1001A800AD28D6280130A2022208FF3A031DDD2817
:1001B800DE289128DF28080083120313A701A6016F
:1001C80002308316031381000730831203139F0044
:1001D800831603138501F03086008B1783120313EF
:1001E8001F149F141F158501FF3086001D30A400C1
:1001F8002408A6008B018B15A50104290429630096
:100208000B1C0729082903290929FF308312031326
:100218008600273081200130831203132C062D0419
:10022800031D1729182904292630A4002408F600DC
:100238002730112083120313AC01AD01A50103146B
:10024800A50D0429042904291028F5018312031394
:1002580005140514051405140510051005100510DE
:1002680005100510051005100510051005100130C2
:10027800F4007408F50720307502031C4429452949
:100288002A2905100800F701A801AA017430A8005E
:100298000230F7000130AA00F70B5029A80B5029AB
:1002A800AA0B50290800F501831203130510013029
:1002B800F4007408F5073C307502031C64296529AD
:1002C800582966290800F701F801F901A801A901D0
:1002D800AA01AB01AC01AD018301E0287308FF005E
:1002E80072088A0071088400700E8300FE0E7E0E6C
:0E02F80009002921572108005721292108005B
:02400E0001FFB0
:00000001FF
